:020000040800F2
:1000000030050020D5000008BD1500083D1400088B
:1000100000000000000000000000000000000000E0
:1000200000000000000000000000000007160008AB
:100030000000000000000000051600080916000876
:10004000E7000008E7000008E7000008E7000008F4
:10005000E7000008E7000008E7000008E7000008E4
:1000600000000000E7000008E7000008E7000008C3
:10007000E7000008E700000800000000E7000008B3
:1000800000000000E7000008000000000000000081
:10009000E700000800000000E7000008E700000893
:1000A000E7000008E7000008E7000008AD1C0008B2
:1000B000E7000008E7000008000000000000000062
:1000C0000348854600F08EF800480047811E00086E
:1000D000300500200448804704480047FEE7FEE75B
:1000E000FEE7FEE7FEE7FEE77D160008C100000818
:1000F00030B50B46014600202022012409E00D46C0
:10010000D5409D4205D31D469540491B2546954047
:1001100040191546521E002DF1DC30BDF0B51FB45C
:100120000646002082B005464024019100901BE065
:10013000019922460F46304600F042F8049A059B8A
:10014000801A994110D310461946224600F028F82B
:10015000361A8F410197224601200021009F00F0AE
:100160001FF838184D4100902046641E0028DFDC3F
:10017000019B00982946324607B0F0BDD2B201E09B
:100180000270401C491EFBD270470022F6E710B5F2
:1001900013460A4604461946FFF7F0FF204610BDF5
:1001A00010B5202A04DB0146203A9140002010BD02
:1001B000914020239C1A0346E3401943904010BD10
:1001C00010B5202A04DB0846203AD040002110BD9B
:1001D0000B46D340D0402024A21A91400843194630
:1001E00010BD0000064C0125064E05E0E36807CC73
:1001F0002B430C3C98471034B442F7D3FFF764FF0D
:100200000C1F00082C1F0008704770B50024014621
:1002100020314A79022A03D00421C163012418E065
:10022000026813680E25AB431360026813685B080D
:100230005B001360436C1C221340012215469D4055
:10024000036C5D604A7100220A71816B002900D045
:100250008847204670BD70B5044600F0CDF80546CD
:10026000601C00D0641C00F0C7F8401BA042FAD309
:1002700070BD0000F8B500230124A2E027469F408E
:100280003A4070D04D68022D01D0122D14D1DD08F6
:10029000AD002D1800952D6A5E07AC46F50E0F26B1
:1002A000AE46AE406546B543AC460E697546AE40B7
:1002B00065462E43009D2E624D68012D05D0022D0E
:1002C00003D0112D01D0122D16D185680326AC461E
:1002D0005D00AE46AE406546B543AC46CE68754659
:1002E000AE4065462E43866046680D79BE43ED06F6
:1002F000ED0F9D403543456006685F000325BD4016
:10030000AE46AE430D79B446AE07B60FBE40654665
:100310002E430660C6687546AE438D68BD403543C2
:10032000C5604D68ED004BD5294D6E6B26436E635D
:100330009E08284DB6007519AC46AD689E07360F6D
:100340000F27B740BD4305273F07B84201D100271B
:1003500015E0214FB84201D1012710E01F4FB842EC
:1003600002D102270BE02BE01D4FB84201D1032739
:1003700005E01C4FB84201D1052700E00627B74031
:100380002F436546AF60184D2E684F689643FF03B4
:1003900000D516432E606E684F689643BF0300D5A4
:1003A00016436E60AE684F689643FF0200D5164351
:1003B000AE60EE684F689643BF0200D51643EE600C
:1003C0005B1C0A681546DD4000D057E7F8BD000009
:1003D00000100240000001400004005000080050DE
:1003E000000C0050001C005000040140002A01D005
:1003F0008161704781627047014800687047000062
:100400001800002070B5024640325378202B1CD1D2
:100410001378012B19D0012313702424547004681D
:1004200025689D432560046825681E03B543256043
:10043000046825680D432560006801681943016060
:10044000202050700020107070BD022070BD70B56B
:10045000024640325378202B1BD11378012B18D041
:10046000012414702423537003681D68A5431D6084
:1004700005682B680F263602B34309021943296029
:100480000068016821430160202050700020107036
:1004900070BD022070BD000070B5040006D0254676
:1004A000403568780026002802D005E0012070BDA4
:1004B0002E70204600F04AF82420687020680168F9
:1004C0004908490001600F216068090688432168D6
:1004D000086121688A680120C00382438A60E1685C
:1004E0000129A16808D0212292021143226891605B
:1004F000E168022902D005E00143F7E70121226803
:10050000C902516021684A680F4B1A434A6021684A
:10051000CA688243CA60616920690843A169090207
:1005200008432168C860216AE069084321680860BF
:100530002068016801221143016066642020687010
:100540002663AE70002070BD0080000210B586B03A
:10055000044614216846FFF718FE114920688842B6
:100560001BD1104CE16A02200143E162E16A0140C3
:10057000032005918002009012200190012002903A
:10058000032003900620049069460748FFF772FE97
:10059000A06B012189050843A06306B010BD0000CF
:1005A000005800400010024000040050024801685A
:1005B000491C0160704700001800002010B5084871
:1005C00000240168402211430160204600F00AF82F
:1005D000002801D0012401E000F01CF8204610BDE5
:1005E0000020024070B5054609487D210024C9005D
:1005F0000068FFF77DFD00F0F9FB002801D0012421
:1006000004E000222946501E00F01AF8204670BD72
:100610001C0000200448416B012211434163816B9F
:10062000020411438163704700100240C106C90EE5
:1006300001208840014908607047000000E100E0A7
:1006400010B500F0BDFF10BDF8B504460078544D5C
:10065000800672D5524E0027403EB06BC00004D4D5
:10066000B06BA9050843B06301274E480168C9056E
:1006700011D40168821511430160FFF7BDFE00909F
:1006800005E0FFF7B9FE0099401A642837D84548BD
:100690000068C005F5D532680321090560680A4085
:1006A0000140914208D08103890F032904D13168A8
:1006B000890301D50120F8BD2A69032109040A40F4
:1006C00022D0084090421FD0207880061CD528698F
:1006D0002A6988430121C9040A432A612A698A4395
:1006E0002A612861C0050FD5FFF786FE009008E05B
:1006F000FFF782FE0099411A2B48814201D903205D
:10070000F8BD28698005F3D561688803800F032848
:1007100005D132680005824301400A4332602869EE
:10072000032261681204114008432861002F04D09D
:10073000B16B012000078143B1632078C00705D069
:10074000E868A168800880000843E8602078800796
:1007500005D5E8680C218843E1680843E860207803
:10076000400706D5E86803218902884321690843C8
:10077000E8602078000706D5E8680321090388436C
:1007800061690843E8602078000606D5E86803211F
:1007900089048843A1690843E8600020F8BD00008F
:1007A000401002400070004088130000F8B50E466B
:1007B00005007DD053480068C007C00FB0420AD280
:1007C0005048016849084900314301600068C0078A
:1007D000C00FB04271D128784B4C800705D5E06836
:1007E000F0218843A9680843E0602878C00752D008
:1007F0006868022817D0032818D02168012818D06B
:100800008905002959DAE168890889000143E16016
:10081000FFF7F2FD69680746022912D003291CD0B0
:10082000012926D033E021688903EAE7216889019C
:10083000E7E74907E5E7FFF7DFFDC11B33488142E2
:1008400023D8E0680007800F0228F4D123E0FFF7E7
:10085000D3FDC11B2D48814217D8E0680007800FE7
:100860000328F4D117E0FFF7C7FDC11B27488142D9
:100870000BD8E0680007800F0128F4D10BE0FFF7E8
:10088000BBFDC11B2148814201D90320F8BDE068AE
:100890000007800FF3D11B480168C907C90FB14297
:1008A0000DD901684908490031430160006800E042
:1008B00003E0C007C00FB04201D00120F8BD287886
:1008C000400706D5E068072109028843E968084324
:1008D000E0602878000707D5E0680721C90288434F
:1008E0002969C9000843E06000F036F8E168084A69
:1008F0000906090F515CC840064908600020FFF74F
:1009000071FEF8BD00200240001002408813000074
:10091000E81E00081C000020044805490068C9685A
:10092000044A4905490F515CC84070471C0000202B
:1009300000100240011F0008044805490068C9680A
:10094000044A8904490F515CC84070471C000020CC
:1009500000100240011F000810B5184AD1680C2091
:10096000084004280BD0082810D00C2810D050685C
:100970000004410F0120C003491C884010BD1068CD
:10098000C00601D50E4810BD0E4810BD0E4810BD62
:1009900088020E4B000F185C0902D368890F491CAE
:1009A000DB0301D5084A05E01268D20601D5044AE6
:1009B00000E0044A5043FFF79BFB10BD00100240CB
:1009C00000093D000024F40000127A00F81E00081F
:1009D000FEB505007ED0FE4CE7680C20E6680740B7
:1009E0000120000406402878C00747D0082F05D012
:1009F0000C2F0AD101200004864206D12068800312
:100A00003CD568680028E5D038E00120696800041A
:100A1000814203D121680143216011E005230122B5
:100A20001B0492049942216802D111432160F1E72D
:100A3000814321602168014000912068904320603B
:100A4000686800280DD0FFF7D7FC009005E0FFF79D
:100A5000D3FC0099401A64287AD820688003F6D520
:100A60000CE0FFF7C9FC009005E0FFF7C5FC00991A
:100A7000401A6428F0D820688003F6D428788007CC
:100A800055D50923E868042F0DD00C2F01D1002E75
:100A900009D000283BD02168994301432160FFF72A
:100AA000ABFC064627E02168490701D5002891D014
:100AB00061681F22120291432A6912021143616088
:100AC0002168994301432160FFF746FFE168090669
:100AD0000A0F00E079E1BF49895CC840BE4908605F
:100AE0000020FFF77FFD002872D120E0FFF784FC93
:100AF000801B0228B0D820684007F7D560681F2106
:100B00000902884329690902084360600FE02068F0
:100B1000400840002060FFF76FFC064604E0FFF746
:100B20006BFC801B022897D820684007F7D42878F0
:100B3000C0065FD5002F0CD0A869002849D02068D6
:100B4000FF21013108432060FFF756FC06462DE0E7
:100B5000C0E02068800502D5A8690028A7D0606899
:100B6000072149038843296A084360606068297F38
:100B70000002000A090608436060286A410B012050
:100B8000C003491C8840E16809060A0F9149895C45
:100B9000C840914908600020FFF724FD002817D1C4
:100BA00028E0FFF729FC801B0228A3D820688005D5
:100BB000F7D56068072149038843296A08436060C4
:100BC0006068297F0002000A09060843606011E09E
:100BD000E1E02168FF20013081432160FFF70CFC38
:100BE000064604E0FFF708FC801B022872D8206844
:100BF0008005F7D42878794E000724D56869002845
:100C0000306910D0012108433061FFF7F5FB0090F7
:100C100005E0FFF7F1FB0099401A02285AD8306925
:100C20008007F6D50FE0400840003061FFF7E4FB95
:100C3000009005E0FFF7E0FB0099401A022849D830
:100C400030698007F6D42878400765D500200290E7
:100C5000A06BC00006D4A06B012109070843A06364
:100C6000012002905E480168C90511D4016882150F
:100C700011430160FFF7C0FB009005E0FFF7BCFBEC
:100C80000099401A642825D855480068C005F5D554
:100C9000FF20AA680130824203D1316901433161EA
:100CA00011E001218902002A07D005231B029A4284
:100CB00003D132690A433261EFE73269824332611C
:100CC000306988433061A86800280FD0FFF794FB93
:100CD000009007E05EE0FFF78FFB0099411A414862
:100CE000814257D830698005F5D50DE0FFF784FBC8
:100CF000009006E0FFF780FB0099411A39488142D5
:100D000048D830698005F5D40298002804D0A06B3B
:100D1000012109078843A063686A002864D00C2F6A
:100D20003ED0012636060228206805D0B043206058
:100D3000FFF762FB05462FE0B0432060FFF75CFB46
:100D4000074604E0FFF758FBC01B022822D82068A2
:100D50008001F7D4E96AA86AE2680843296BFD2399
:100D60001B049A4311430843E0602068304320602D
:100D7000FFF742FB054604E0FFF73EFB401B02285D
:100D800008D820688001F7D52EE0FFF735FB401B1F
:100D9000022801D90320FEBD20688001F5D423E09C
:100DA0000128F8D0E06801210904AA6A01409142B3
:100DB0000BD10F218904EA6A0140914205D1032138
:100DC00089050840296B88420ED00120FEBD000035
:100DD00000100240E81E00081C00002040100240E5
:100DE00000700040881300000020EFE7094910B5AB
:100DF000401E884201D9012010BD074C60610321CB
:100E0000081F00F0DDFB0020A0610720206100200A
:100E100010BD0000FFFFFF0000E000E0F0B502465B
:100E20002032137E012B15D001271776022353762B
:100E300005686C68AB687026B4430E684968264341
:100E40008024A34319436E600068816057760020B8
:100E50001076F0BD0220F0BD10B586B00446142116
:100E60006846FFF792F90D492068884213D10C4873
:100E7000C26A02210A43C262C06A01910840059019
:100E800010200090002002900390042004906946F6
:100E90000448FFF7EFF906B010BD00000014014050
:100EA0000010024000040050F8B506460446203603
:100EB000307E0D4601280DD001203076022070765C
:100EC0000427002A08D0042A16D0082A2AD00C2A7F
:100ED0004DD137E00220F8BD206800F032FC2068D8
:100EE000816908221143816120688169B943816168
:100EF00020688169EA6812E0206800F03AFC206806
:100F000082690121C9020A43826120688169012244
:100F100092029143816120688169EA68120211435B
:100F2000816124E0206800F03DFC2068C26908214E
:100F30000A43C2612068C169B943C1612068C169BF
:100F4000EA6812E0206800F048FC2068C1690122CC
:100F5000D2021143C1612068C269012189028A431A
:100F6000C2612068C169EA6812021143C1610120AF
:100F7000707600203076F8BD70B5040005D02546A7
:100F80002035687E002802D006E0012070BD0020D8
:100F90002876204600F00AF802206876211D206895
:100FA00000F096FB01206876002070BD00680449BF
:100FB000884204D10348416B2022114341637047AA
:100FC000001401400010024010B5044600680122E0
:100FD00000F0AAFB206881684907490F062903D061
:100FE0000168012211430160002010BD7047704765
:100FF000F8B502680446D0691168936805072D0F9B
:101000005BD0DD07ED0FFF2621360E402E4367D063
:10101000C60706D0CE0504D501261662E26F32431C
:10102000E267870702220426002F06DADF0704D0D2
:1010300027683A62E76F3743E767470706D5DB075C
:1010400004D023681E62E36F1343E367020709D5E8
:1010500020220A402A4305D0236808221A62E36F3F
:101060001343E367E26F002A2FD0800606D5880677
:1010700004D5216E002901D020468847E06F216801
:101080008968490601D4000724D5204600F060FC99
:1010900020688168490619D58168402291438160A2
:1010A000E06E002812D020498163E06EFFF7ADF8B2
:1010B00000280AD0E06E816B06E0850610D58D060B
:1010C0000ED5216E1CE020468847F8BD2046FFF76C
:1010D0008EFFF8BD2046FFF78AFF0020E067F8BDCD
:1010E000C50208D55B0206D5012000051062204626
:1010F000FFF77CFFF8BD030605D50B0603D5616E2F
:101100000029E0D1F8BD4006FCD54806FAD51368A1
:10111000204640218B4313602021616700216166D6
:1011200000F08BF9F8BD00003D19000810B504006F
:1011300003D0606F002802D007E0012010BD00211D
:1011400070200155204600F027F8242060672068B1
:101150000168490849000160204600F061FC01284F
:10116000ECD0606A002802D0204600F051FB2068D5
:1011700041680922D20291434160206881682A2295
:10118000914381602068016801221143016020467B
:1011900000F0A4FB10BD000010B586B00446142179
:1011A0006846FEF7F2FF15492068884224D11448AA
:1011B000416B0122920311434163C16A0122114331
:1011C000C162C06A69461040059003204002009049
:1011D000022001900020029003200390042004903C
:1011E00005200007FFF746F8002211461B20FFF7F5
:1011F00027FA1B20FFF71AFA06B010BD003801408D
:1012000000100240F0B5836F202B54D100290AD082
:10121000002A08D08568DC01A54206D10369002BAD
:1012200003D1CB0701D00120F0BD034660331E7C03
:10123000012E40D001261E744165014640310A83CB
:101240004A830022FF260266A54204D10569002DCB
:1012500013D11A4D0AE07F27002D09D00126360749
:10126000B5420CD10569002D05D03F258D8307E0DF
:101270000569002D01D08F8302E08E8300E08A8310
:10128000C2672221816701688D68012635438D6020
:101290008168A14202D1016900290AD0084901668A
:1012A0001A7400680168FF22213211430160002096
:1012B000F0BD0449F3E70220F0BD0000FF0100008B
:1012C000C91900087119000870B5224EF07803287A
:1012D00007D03146322305220C391F4800F046F86A
:1012E00070BD1C4C30790125103C012808D12168C3
:1012F0002046491C09302160457018A000F0DEFC32
:101300003079022805D1216814A0491E216000F01F
:10131000D5FC3079032804D14D2110A0216000F0C4
:10132000CDFC3079042804D12E210CA0216000F0DE
:10133000C5FC3079052804D1294608A0256000F0B5
:10134000BDFC30790628CBD1002104A0216000F03B
:10135000B5FC70BD10000020AC000020445554596D
:10136000204359434C453A25640D0A00FFB5044615
:10137000406F83B017460D4620285CD1002D0AD05F
:10138000002F08D0A168C001814207D12069002840
:1013900004D1E80702D0012007B0F0BD204660303C
:1013A0000290007C012846D002980121017400209F
:1013B000E06721206067FFF71FF82646403601905E
:1013C000378277820120A1680003814202D120691F
:1013D000002802D02F46002511E000270FE0002250
:1013E0008021204600F030FC002815D1002F15D0B8
:1013F0002168387888627F1C708A401E7082708AEB
:10140000019B002806980090E9D100224021204647
:1014100000F01AFC002808D00320BDE728882168C6
:10142000C005C00D8862AD1CE6E720206067029908
:1014300000200874B0E70220AEE77047FEE7000026
:10144000F0B587B014216846FEF79FFE1848C26ABF
:1014500002210A43C262C26A0A400592C16A01259A
:101460002943C162C06A032428400526E4023607E6
:101470000590002221463046FEF7B8FF0D4F0022AE
:1014800060213846FEF7B2FF0094002401950294D3
:10149000694630460394FEF7EDFE6020009002940A
:1014A0006946019503943846FEF7E4FE07B0F0BDA7
:1014B000001002400004005010B5134811490160AB
:1014C0001249416000218160016141618161012215
:1014D000C161C2600162FEF7DFFF002801D0FEF7A4
:1014E00093FE00210848FEF78DFF002801D0FEF78B
:1014F0008BFE00210448FEF7AAFF002801D0FEF76A
:1015000083FE10BD005800402400002009050000A3
:1015100010B586B0002405941948049400940194F1
:1015200002941649039401601321846041600461B0
:1015300063214461C160FFF71FFD002801D0FEF761
:1015400063FE049404A90E480594FFF767FC002885
:1015500001D0FEF759FE6020009001940294002211
:10156000694603940648FFF79FFC002801D0FEF768
:101570004BFE0348FFF770FC06B010BD001401409D
:101580007000002010B50C480A490160E1214902B1
:10159000416000218160C16001618161C1610C22F3
:1015A000016242614162FFF7C1FD002801D0FEF7F0
:1015B0002BFE10BD00380140AC0000207047000039
:1015C0008307FF22DB0E9A408907090E9940002805
:1015D0000BDA0007000F0838830808489B0018182A
:1015E000C36993430B43C3617047830804489B005E
:1015F0001B181868904308431860704700ED00E01E
:1016000000E400E07047704710B5FEF7CFFF10BD53
:1016100030B599B034216846FEF7B7FD14210DA806
:10162000FEF7B3FD1C2112A8FEF7AFFD12480168BA
:101630000322D2029143C214891801600220009053
:101640000024102009940125049003956846FFF7B3
:10165000BFF90F200D90A0200F900E95109400213F
:1016600011940DA8FFF7A2F812A812951494FEF792
:10167000EBFF19B030BD0000007000401048016859
:10168000821511430160C1680E4A1140C1600168B2
:101690000D4A114001608168490849008160016874
:1016A0000122920491430160C168FD22120491431A
:1016B000C160002101610549C003886070470000D6
:1016C000001002400C40FF88F6FFF6FE00ED00E03F
:1016D00070B5026801239B07114C124D984203D04C
:1016E000A04201D0A84203D17026B2434E683243D3
:1016F000984203D0A04201D0A84204D103231B0288
:101700009A43CB681A4380239A430B691A430260B9
:101710008A68C262096881620121416170BD00006E
:10172000000801400014014010B5CB06DB0E01217A
:10173000046A99408C430462016A9A401143016231
:1017400010BD30B5026A520852000262026A456852
:1017500083697024A3439C080B68A40023430224DC
:10176000A2438C6845601443836149684163046205
:1017700030BD30B5026A10239A430262036A45689D
:10178000826973242402A2430C6824021443202299
:1017900093438A68456012011A43846149688163F2
:1017A000026230BD30B5026AFF2301339A43026200
:1017B000026A4568C3697024A3439C080B68A400AF
:1017C000234301246402A2438C684560240214432D
:1017D000C3614968C163046230BD30B5026A012348
:1017E0001B039A430262036A4568C2697324240298
:1017F000A2430C68240214430122520393438A68D3
:10180000456012031A43C46149680164026230BD35
:1018100010B5818CC90707D001684A6801235B04B1
:101820009A43836A1A434A60818C890707D5016805
:101830004A6801231B049A43C36A1A434A60818C95
:10184000490707D501684A6801239B049A43036B43
:101850001A434A60818C090707D501684A68012349
:10186000DB039A43436B1A434A60818CC90607D550
:101870000268916801231B039943836B19439160AC
:10188000818C890607D501688A6801235B039A4326
:10189000C36B1A438A60818C490612D503685A6863
:1018A00001210905046C8A4322435A60026C8A4272
:1018B00007D10268516803235B059943436C1943C0
:1018C0005160818C090607D501684A680123DB0451
:1018D000806C9A4302434A6010BD0000F8B50026B0
:1018E0000446C667FEF788FD054620680068124F6B
:1018F000000709D501212B46002249052046009703
:1019000000F0A2F900280DD12068006840070BD52F
:1019100001212B46002289052046009700F094F90A
:10192000002801D00320F8BD20206067A067603444
:1019300026740020F8BD0000FFFFFF0110B5806A8B
:101940000022014640314A834A82FFF750FB10BD16
:1019500001680A68FF2321339A430A6001688A6894
:10196000520852008A602021816700210166704779
:1019700010B5014640318B8B846F0268222C04D055
:10198000906908210843906110BD526A446D1A4065
:101990002280426D921C42654A8B521E4A83498BBB
:1019A0000029F1D101680A68FF2321339A430A60B4
:1019B00001688A68520852008A60202181670021EC
:1019C0000166FFF781FC10BD10B5014640318B8BDD
:1019D000846F0268222C04D090690821084390612A
:1019E00010BD526A1A40436D1A70426D521C426516
:1019F0004A8B521E4A83498B0029F1D101680A683B
:101A0000FF2321339A430A6001688A685208520012
:101A10008A602021816700210166FFF755FC10BD17
:101A2000F8B504462669A268E76932436669102062
:101A300000253E432368324378491E68784F3E4074
:101A400016431E6023685A6803263603B243E668CD
:101A500032435A602368A2698B4201D0266A32431E
:101A60009E680B273F02BE4316439E606D4E23685F
:101A70006D4AB3420CD1D2689207920F06D0012A68
:101A800038D0022A34D0032A20D11EE001201DE0E4
:101A9000664EB3420AD1D2680C26324026D0042AC0
:101AA00028D0082A24D00C2A10D10EE08B420DD168
:101AB000D66803229202164018D001229202B61A6A
:101AC00018D0B61A14D0964200D10820564A0126E2
:101AD000403A574FF6038B4236D100280CD00228EB
:101AE0000DD0042812D008281FD11CE00020EDE7FB
:101AF0000220EBE70420E9E7FEF70EFF08E010689C
:101B0000C00601D5384605E04A4803E0FEF724FF49
:101B1000002873D0626851005118814205D8110322
:101B2000814202D303E03046F4E7012566E0010E6E
:101B300006025008002330185941FEF7EFFA03213E
:101B40000902411A3C4A55E0E169B14232D1030031
:101B500000F0C4F809070A0D06250606062B060044
:101B6000E3E7FEF7D9FE1CE0FEF7E6FE19E0106899
:101B70006168C00602D54808304A01E0304A48088A
:101B80008018FEF7B5FA80B201462E4A103991420C
:101B9000CBD8511C01400007400F08432CE0FEF752
:101BA000DBFE616840004A08EAE7616801224808F4
:101BB0001204E5E7030000F091F809070A0D062674
:101BC0000606062C0600B0E7FEF7A6FE1DE0FEF7AF
:101BD000B3FE1AE010686168C00602D54808C01953
:101BE00002E014484A081018FEF782FA80B2014653
:101BF000144A1039914298D82168C86000202066A4
:101C000060662846F8BDFEF7A7FE61684A0880189E
:101C1000EAE7616848088019E6E7000000480040EC
:101C2000F369FFEF003801404010024000440040DB
:101C300000093D000024F400FFFC0F0000127A00B0
:101C40000048E801EFFF0000FFB581B017460E46DF
:101C500004460A9D09E0681C07D0FEF7CDFB0499F5
:101C6000401AA8420CD8002D0AD02068C16930461D
:101C7000884318D00020B842EDD0002005B0F0BD58
:101C800020680168FF22A1329143016020688168C9
:101C900049084900816020206067A0670020603407
:101CA00020740320EAE70120E5E7000010B50248B0
:101CB000FFF79EF910BD0000AC0000200FB410B576
:101CC00003A9044B044A029800F024F810BC08BC95
:101CD00004B01847651E00082000002030B4744688
:101CE000641E2578641CAB4200D21D46635D5B0018
:101CF000E31830BC184702E008C8121F08C1002AC8
:101D0000FAD170477047002001E001C1121F002A7C
:101D1000FBD17047FFB58DB00446002506E02528AD
:101D20000AD0109A0F999047641C6D1C20780028E7
:101D3000F5D1284611B0F0BD00270121484A00978F
:101D400000E00743641C23780846203B984010427B
:101D5000F7D120782E2817D1042007436078641C1F
:101D60002A280CD10E98641C02C800910E900BE03A
:101D700000990A22514330394018641C00902078A1
:101D8000014630390929F3D920780028D1D06428B8
:101D900008D0692806D075281ED0109A0F99904750
:101DA0006D1C5BE00A200E99019001C90E9100287C
:101DB00002DA40422D2102E0390504D52B216A4682
:101DC0001172012103E0F90704D02021F7E70BAEDF
:101DD0000B910DE00021FAE70A200E99019001C94C
:101DE0000E91F7E70199FEF783F93031761E3170D5
:101DF0000028F7D103A8801B20300190780701D577
:101E0000009801E0012000900199884201DD401A0C
:101E100000E000200027009006E002A8109AC05DB4
:101E20000F9990476D1C7F1C0B988742F5DB04E0EF
:101E3000109A30200F9990476D1C0099481E009011
:101E40000029F5DC05E03078109A761C0F99904750
:101E50006D1C0199481E01900029F4DC641C65E7A3
:101E60000928010001B5044B012269460348FFF728
:101E70007DFA009808BD0000FFFF0000AC000020C4
:101E80001FB5FEF79BFBFFF7C3FBFFF7D9FAFFF780
:101E900013FBFFF777FBFFF73BFB00210F48FFF732
:101EA00093F800240E4D60260D49072210310D488D
:101EB000FFF7A8F96420FEF7CEF92888029480B2D3
:101EC000019000226946009603940448FEF7ECFF57
:101ED00000210248FFF778F8E6E7000070000020D4
:101EE00000000020AC000020000000000000000006
:101EF0000102030406070809030406080C10182051
:101F00003000000000010203040000002C1F000844
:101F10000000002024000000F61C0008501F0008EC
:101F2000240000200C050000061D00080000000031
:101F3000FF0102030DFF0100000D00000000000082
:101F40000000000000000000000020000000000071
:04000005080000C12E
:00000001FF
